:020000040800F2
:100000000004022001020008E10C0008E10C0008D5
:10001000E10C0008E10C0008E10C0008E10C00080C
:10002000E10C0008E10C0008E10C00082D2F00088D
:10003000E10C0008E10C0008E10C0008E10C0008EC
:10004000E10C0008E10C0008E10C0008E10C0008DC
:10005000E10C0008E10C0008E10C0008E10C0008CC
:10006000E10C0008E10C0008E10C0008E10C0008BC
:10007000E10C0008E10C0008E10C0008E10C0008AC
:10008000E10C0008E10C0008E10C0008E10C00089C
:10009000E10C0008E10C0008E10C0008E10C00088C
:1000A000E10C0008E10C0008E10C0008E10C00087C
:1000B000BD260008E10C0008E10C0008E10C000876
:1000C000E10C0008E10C0008E10C0008E10C00085C
:1000D000E10C0008E10C0008E10C0008E10C00084C
:1000E000E10C0008E10C0008E10C0008E10C00083C
:1000F000E10C0008E10C0008E10C0008E10C00082C
:10010000E10C0008E10C0008E10C0008E10C00081B
:10011000E10C0008E10C0008E10C0008E10C00080B
:10012000E10C0008E10C0008E10C0008E10C0008FB
:10013000E10C0008E10C0008E10C0008E10C0008EB
:10014000E10C0008E10C0008E10C0008352400086F
:10015000E10C0008E10C0008E10C0008E10C0008CB
:10016000E10C0008E10C0008E10C0008E10C0008BB
:10017000E10C0008E10C0008E10C0008E10C0008AB
:10018000E10C0008E10C0008E10C0008E10C00089B
:10019000E10C0008E10C0008E10C0008E10C00088B
:1001A000E10C0008E10C0008E10C0008E10C00087B
:1001B000E10C0008E10C0008E10C0008E10C00086B
:1001C000E10C0008E10C0008E10C0008E10C00085B
:1001D000E10C0008E10C0008E10C0008E10C00084B
:1001E000E10C0008E10C0008E10C0008E10C00083B
:1001F000E10C0008E10C0008E10C0008E10C00082B
:1002000072B6374880F3098836484EF60851CEF268
:100210000001086040F20000CCF200004EF634719C
:10022000CEF200010860BFF34F8FBFF36F8F40F233
:100230000000C0F2F0004EF68851CEF200010860D6
:10024000BFF34F8FBFF36F8F4FF00000E1EE100A46
:100250004EF63C71CEF200010860062080F314884F
:10026000BFF36F8F00F0E2FC02F068FA4FF05530F8
:100270001D491E4A91423CBF41F8040BFAE71C4954
:10028000174A91423CBF41F8040BFAE719491A4A50
:100290001A4B9A423EBF51F8040B42F8040BF8E7A0
:1002A00000201749174A91423CBF41F8040BFAE776
:1002B00000F0FCFC02F044FA134C144DAC4203DA9B
:1002C00054F8041B8847F9E700F0ACF8104C114DC6
:1002D000AC4203DA54F8041B8847F9E700F0E4BCA9
:1002E0000008022000000008000002200004022094
:1002F00000040220A03A0008000802204C08022056
:1003000050080220D818022000020008000200084D
:1003100000020008000200082DE9F04F2DED108AC0
:10032000C1F80CD0D0F80CD0BDEC108ABDE8F08F2D
:10033000002383F311882846A047002000F020FF07
:1003400000F07CFE00DFFEE790F800F06DE902456A
:1003500020F007016FF0000C10F0070491F820F076
:1003600040F049804FF000046FF00700D1E900230E
:1003700091F840F000F1080082FA4CF2A4FA8CF2F5
:1003800083FA4CF3A2FA8CF34BBBD1E9022382FA35
:100390004CF200F10800A4FA8CF283FA4CF3A2FAB2
:1003A0008CF3E3B9D1E9042382FA4CF200F108009E
:1003B000A4FA8CF283FA4CF3A2FA8CF37BB9D1E95C
:1003C000062301F1200182FA4CF200F10800A4FAA0
:1003D0008CF283FA4CF3A2FA8CF3002BC6D0002ADD
:1003E00004BF04301A4612BAB2FA82F2FDE802459E
:1003F00000EBD2007047D1E9002304F00305C4F1FB
:1004000000004FEAC50514F0040F91F840F00CFA13
:1004100005F562EA05021CBF63EA050362464FF078
:100420000004A9E71D4C1E4808B501F045F8214617
:100430001B4801F06DF823681A48DA6ED2F80438C8
:1004400043F00203C2F8043800F0A0FE1649206809
:1004500001F078F92368DA6ED2F8043823F0020349
:10046000C2F80438114B782119706FF07F01002217
:1004700059721E215A709A70DA701A715A719A71F3
:10048000DA711A729972DA7200F006FB41F2883062
:1004900000F0B8F800F044F8F8E700BF5039000861
:1004A0009011022040420F00B83900085008022085
:1004B00008B500F0C3FAA0F120035842584108BD26
:1004C0000248C3680BB100F0D7BC70475C0802203B
:1004D00010B50F4CFFF7F4FF00230E4A0E484FF4FF
:1004E0007A7100F08DFC236813B12368013B23600F
:1004F000636813B16368013B6360084B1B7833B9D1
:10050000636823B9022000F075FB3223636010BDDD
:10051000740D0220D10400085C080220700802203B
:100520002DE9F041314C236801335CD0304E314B22
:1005300032689A4257D9304B9B6803F1006303F548
:10054000C0339A424FD22D4B0220187000F050FB5E
:10055000202383F31188FFF7B3FF002282F3118871
:10056000274B1C6025683668BFF34F8FBFF36F8F32
:10057000083BC3F88420BFF34F8FD3F8802059691C
:10058000C2F3C90421F48031C2F34E3259615201E1
:10059000A70743F6E07E02EA0E08384621460139F5
:1005A00048EA000CB1F1FF3FC3F874C200F14040CB
:1005B000F5D1203A12F1200FEDD1BFF34F8FBFF3E9
:1005C0006F8FBFF34F8FBFF36F8F5A6922F40032E2
:1005D0005A610022C3F85022BFF34F8FBFF36F8FD1
:1005E00085F308883047BDE8F08100BF008001082E
:1005F00004800108FF7F01085008022070080220D3
:1006000008ED00E02DE9F04FC44FDFF82C83BC6803
:1006100000268FB00546C8F80C60202383F31188AC
:10062000FFF74EFF3346BE4A4FF47A71404600F062
:10063000E7FB86F31188DFF80493B84633460DB123
:10064000C9F80050B74EC9F8043033704FF0FF3787
:10065000012000F0CDFA002D00F0B881D9F800306B
:10066000002B40F0B3810FB0BDE8F08F0220FFF700
:100670001FFF00283BD112238DF8243013230221C1
:1006800009A88DF8253000F0F7F9E1E74FF47A700A
:1006900000F0D4F9B0F1000BEDDB0220FFF708FF0A
:1006A0000028E8D00BF1FF300428E4D8DFE800F0A0
:1006B00003080D10130005230993042109A801E084
:1006C0009648042100F0D8F911E004219648F9E792
:1006D00004219648F6E71C25284600F0F9F9043570
:1006E0000990042109A800F0C7F92C2DF4D1122398
:1006F0008DF824300221102309A88DF8253000251B
:1007000000F0BAF9A4E70220FFF7D2FE0028B2D029
:100710000220307000F06CFA4FF0000B5FFA8BFA99
:10072000504600F0EBF90BF1010B044618B15046AE
:1007300000F0F4F9F2E701230220337000F056FADA
:10074000D8F808309C4207D2204600F0C1F90130A9
:1007500040F035810434F3E700243470C9F80440D4
:10076000C5E70220307000F043FA322000F066F94D
:10077000B0F1000BFFF67FAF1BF003037FF47BAFFC
:10078000D8F808100BEB04028A423FF674AFBBF5B1
:10079000807F3FF670AF664A9A46DA4501920FDADB
:1007A0004FF47A7000F04AF9039003990029FFF69C
:1007B00062AF019A03990AF802100AF1010AECE704
:1007C000C820FFF775FE00283FF455AF24B9584BF9
:1007D0004FF0FF321F681A60554B2BF0030BA344F8
:1007E000A3EB040AA34500F0EF805AF8041020465A
:1007F00000F074F9204600F06BF95AF8042090429A
:1008000040F0DD800434EDE70220FFF751FE0028C0
:100810003FF431AF4FF0000B5D46D8F808309B45F0
:1008200034D2BBF1000F14D17A1C12D00997414980
:100830004B689BB1002209A8135C6B40DBB201320C
:1008400051F82330042A83EA1525F5D10BF1040B66
:10085000E3E7584600F03CF90990E8E71A4608201B
:1008600012F0010F4FEA52021FBF82F06D4282F474
:10087000380282F4034282F020020138F0D141F8BC
:1008800023200133B3F5807FE8D1D3E70EA80421FC
:1008900040F8285D16E74FF0000B0DF1240A6420A4
:1008A00000F0CCF80028FFF6E6AE0BF80A000BF1DA
:1008B000010BBBF1040FF2D10220DDF824A0FFF7F9
:1008C000F7FD00283FF4D7AE504600F02FF90EABED
:1008D00043F8240D04211846F4E64FF0000B0DF107
:1008E000240A642000F0AAF80028FFF6C4AE0BF832
:1008F0000A000BF1010BBBF1040FF2D1099B01932C
:100900000220FFF7D5FD019B00283FF4B4AE184646
:1009100000F01AF90EAB43F8200DDBE75008022077
:10092000D104000870080220540802205808022050
:1009300074080220740902205C080220740D022051
:100940000220FFF7B5FD00283FF495AE00F002F954
:100950000EAB43F81C0DBDE70220FFF7A9FD0028F0
:100960003FF489AE09A9142000F0FAF805460EA854
:10097000042140F8185D00F07FF829469EE64FF408
:100980007A70FFF795FD00283FF475AE7B1C0DD102
:1009900012238DF8243009A8102302218DF8253068
:1009A00000F06AF8244800F0F1FB5CE639460020CC
:1009B00000F094F8002000F08BF88742E8D0122372
:1009C0008DF8243011235AE65C4690E6002000F0B2
:1009D00035F80390039B002BFFF63DAE012000F09D
:1009E00005F9039B213B102B3FF632AE01A252F8D2
:1009F00023F000BF6D0600088D06000807070008F9
:100A00005106000851060008510600086307000857
:100A1000510600080908000897080008DB080008CC
:100A2000410900085106000859090008510600084C
:100A30007F090008EF060008A086010073B50D4D80
:100A400002A9002301F8013D2B684FF47A74DE6996
:100A5000012204FB00F32846B047012806D02046B7
:100A600000F094FB4FF0FF3002B070BD9DF807001E
:100A7000FAE700BF9011022030B4054C23689D694D
:100A8000044B0A46AC460146204630BC604700BFD6
:100A900090110220A0860100F8B501F0C1FF094CB9
:100AA000094E0A4F2070002530682378834207D909
:100AB00001F0B0FF336805440133BD423360F3D920
:100AC000F8BD00BF800D02207C0D0220FF7F0100D9
:100AD00000F1006000F5C0300068704707B502AB58
:100AE00000F1006043F8041D0422194600F5C030EF
:100AF00001F0D0FF03B05DF804FB0000054B1A685D
:100B0000054B1B781344834202D9104401F082BF85
:100B1000002070477C0D0220800D0220024B1B68D4
:100B2000184401F07FBF00BF7C0D022010F00303CA
:100B300008D1B0F5806F05D800F10050A0F5712004
:100B40000068704700207047014BC058704700BFD5
:100B500020F4F01F014B1868704700BF002004E02C
:100B6000F0B5204B1E68204B1F885D6893F9084044
:100B7000C6F30B02BA424FEA164622D09F89BA4208
:100B800021D01F8BBA4206D102220C2404FB02336F
:100B90005D6893F90840B6F5805F16D041F2010315
:100BA0009E4208BF5A24421E0A44013D0B4693420E
:100BB00015D215F9016F581C4EB1034600F8016CAF
:100BC000F5E70022E1E70122DFE74124EBE72C25EE
:100BD00082421D7001D9981C5C70401AF0BD184605
:100BE000FBE700BF002004E000080220704700007F
:100BF000704700007047000010B50023934203D0F7
:100C0000CC5CC4540133F9E710BD000010B50138C5
:100C100010F9013F0A462BB192F900409C4201F1C4
:100C20000101F5D092F90000181A10BDF0B5BFF31C
:100C30004F8FBFF36F8F1B4B0021C3F850125A69BF
:100C400042F400325A61BFF34F8FBFF36F8FC3F886
:100C50008410BFF34F8FD3F88020C2F3C904C2F3CE
:100C60004E325201A50743F6E07602EA060E284608
:100C700021464EEA00070139C3F860724F1C00F1AB
:100C80004040F6D1203A12F1200FEED1BFF34F8F42
:100C90005A6942F480325A61BFF34F8FBFF36F8FAE
:100CA000F0BD00BF00ED00E0FEE70000084A094B80
:100CB00009498B4204D3094A0021934205D3704766
:100CC00052F8040F43F8040BF3E743F8041BF4E76E
:100CD000E83A0008D8180220D8180220D8180220B4
:100CE0001EF0040F0CBFEFF30880EFF30980816959
:100CF000004A1047FD0C000870470000204B0268B6
:100D00001A60204B42681A601F4B82681A601F4BA2
:100D1000C2681A601E4B02691A601E4B42691A6053
:100D20001D4B82691A601D4BC2691A601C4B1D491C
:100D30001A681D4B1A601A68120A0A701A681B4B4F
:100D40001A701B4B1A681B4B1A601B4B1A681B4B03
:100D50001A601B4B1A681B4B1A601B4B1A681B4B03
:100D60001A601B4B1A681B4B1A601B4B5A6A1B4BB1
:100D70001A601B4B1B68DB0701D500BEFEE7FEE7D0
:100D8000B40D0220B80D0220C00D0220C40D0220B7
:100D9000BC0D0220A80D0220AC0D0220B00D0220D7
:100DA00028ED00E08C0D0220900D0220A00D022005
:100DB0002CED00E0980D022030ED00E0940D0220B3
:100DC0003CED00E0840D022034ED00E09C0D02209B
:100DD00038ED00E0880D022000ED00E0A40D0220B7
:100DE000F0ED00E0054B03F11C02DA611A624FF0EE
:100DF000FF325A6200229A62704700BFC80D02207B
:100E0000F8B503614FF08043C2605C6A194B1A4623
:100E1000022952F81C5F38BF0221954206461F4640
:100E20000AD1D86118629C6205604560816008192A
:100E3000BDE8F84000F062BC986AAB68241A0C194F
:100E400002D3E41A2D6804E09C4202D2204400F050
:100E500063FCAB689C42F4D86B68736035601E60BD
:100E60006E60B460A9684FF0FF33091BA9607B6214
:100E7000F8BD00BFC80D022010B41B4C234653F828
:100E80001C1F814210D0416802680A6002685160EC
:100E90009A424FF00001C16003D0936881680B440F
:100EA00093605DF8044B70470A68E26100209A4243
:100EB0005360C86003D15DF8044B00F027BC936811
:100EC0008868034493604FF08042506AA26A821A95
:100ED0009342E6D99B1A022B2CBFC01802305DF852
:100EE000044B00F019BC00BFC80D0220034B0022C8
:100EF0001B605B609A601B615B617047C80D0220DC
:100F0000002380F820308268054B1B689968914265
:100F1000FBD25A680360426010605860704700BF9F
:100F2000C80D022008B5202383F3118890F82020F3
:100F30000023072A07D8DFE802F00C060604130F87
:100F40000613426A13604FF0FF334362FFF7D8FF86
:100F5000002383F3118808BD426A936801339360CC
:100F600090E80C001A6002685360ECE7002380F8F8
:100F700020308268054B1B6899689142FBD85A68FB
:100F80000360426010605860704700BFC80D0220C7
:100F9000064B996981F82000186802681A6053604E
:100FA0009861012380F82030FFF7B6B9C80D022000
:100FB00030B54B1C87B005460A4C10D0A3690A4ACD
:100FC00001A8FFF71DFF2846FFF7E2FF049B13B1BE
:100FD00001A8FFF751FFA369586A07B030BDFFF7BA
:100FE000D7FFF8E7C80D0220250F000838B50C4DD3
:100FF0004162AB6981689A689142044603D8BDE8B2
:101000003840FFF77DBF1846FFF77AFF0123AC6138
:1010100084F8203001462046BDE83840FFF77CB90F
:10102000C80D0220044B1A689B6990689B6898421F
:1010300094BF002001207047C80D022010B5094C54
:101040002368A0691A6822605460012283F8202076
:10105000A361FFF78BFF0146A069BDE81040FFF7D1
:101060005BB900BFC80D022008B5FFF7DBFF18B160
:10107000BDE80840FFF7E2BF08BD00008260C26320
:10108000012280F822200C4A816110B55169026169
:10109000022480F820400024416180F821408463CC
:1010A00044630861506100F12802826200F12C0261
:1010B000C262026310BD00BFC80D0220884200D387
:1010C000704700F8012BF9E78368426843F82C2C3D
:1010D000A3F1AC0243F83C2C026943F86C2C426942
:1010E00043F8682C044A43F84C2C0168C268A3F109
:1010F0004800FFF7C3BF00BF3103000808B5FFF782
:10110000E3FFBDE80840FFF7FBBE000010B58268B2
:10111000436855219A420DD8202383F31188FFF7A5
:10112000D3FF00210446FFF761FF002383F31188FA
:10113000204610BD03F8011BECE7000038B50F4B4B
:101140009C69606204F12805A06AA84210D194F855
:10115000223043B994F821309B0704D16369226996
:101160001A61226953610F20BDE83840FFF710BFB4
:101170000368A362FFF7C4FEE6E700BFC80D0220C4
:10118000202383F31188FFF7D9BF000008B501467B
:10119000202383F311880820FFF70AFF002383F33D
:1011A000118808BD10B5054CA3690360586203207F
:1011B000FFF7EEFEA369586A10BD00BFC80D0220FC
:1011C00003682BB10022026059621846FFF798BEEF
:1011D0007047000049B1064B42689B6918605A602D
:1011E000136043600420FFF7E3BE4FF0FF30704709
:1011F000C80D02200368984206D01A680260506049
:1012000059621846FFF77CBE7047000038B50446A7
:101210000D462068844200D138BD036823605C60BD
:101220004562FFF76DFEF4E70448054B03600023B9
:101230008360C360103001F0A1BD00BF400E0220EA
:10124000192F0008083A0023D20803608160C360A8
:101250000B604A60103001F091BD00002DE9F84F9D
:10126000384E002818BF0646082A38BF082206F163
:1012700010089146CC1D40460F46E40801F0C4FD1D
:1012800009F1FF3A06F10801C9F1000B0B683BB9FF
:10129000404601F0C3FD3368002B48D100242DE007
:1012A00003F1080C5A680CEB0A0505EA0B0502F17C
:1012B000010EA5F1080003EBCE0E704535D2AEEB62
:1012C0000505ED10AC4230D883421AD2A0EB0C0CCD
:1012D0004FEAEC02AC425A6009D2611C00EBC10239
:1012E000E443254455601C6840F831401A600446C8
:1012F000476044F8086B404601F090FD2046BDE889
:10130000F88F94421A6802D10A601846EFE7013458
:1013100003EBC40543F8342005F10802AEEB020EDE
:101320004FEAEE026A600D60EFE71946AEE7601C17
:101330004946C00098470028B0D080E8C00000F1BE
:101340000804DBE7400E0220F8B550F8043C50F8E2
:10135000086C0733DB0806F10807103640F8043C38
:101360000446A0F10805304601F04EFD3B46BB4265
:101370001A6801D0AB4229D20AB1954226D244F86C
:10138000082C1D6054F8042C54F8080C013205EBAD
:10139000C201814207D14968114444F8041C55F840
:1013A000322044F8082C5868411C03EBC1018D42DF
:1013B00007D154F8042C013202445A6054F8082C26
:1013C0001A603046BDE8F84001F028BD1346CEE76C
:1013D00013B5446BD4F88C341A681178042916D1EB
:1013E000217A022913D11979128901238B401342E2
:1013F0000DD101A904F1440001F0F4FE024630B120
:10140000D4F88C44019B2179206800F0EBF902B0FC
:1014100010BD00000C3001F063BE00004FF0FF3340
:101420000C3001F05DBE0000443001F047BF000009
:101430004FF0FF33443001F041BF00000C3001F0A9
:1014400031BE00004FF0FF310C3001F02BBE000028
:10145000443001F013BF00004FF0FF32443001F080
:101460000DBF0000D0F88C2438B513681978042912
:10147000054601D0012038BD017A0229FAD112793E
:101480005C89012090400440F4D105F10C0001F08A
:10149000C3FD02460028EDD0D5F88C544FF480737C
:1014A0002868697900F08CF9204638BD406BFFF759
:1014B000D9BF0000704700007FB50346114A43F8CA
:1014C000042B0125436002260F4B0572044602904F
:1014D000019300F17C02294600964FF480730C3092
:1014E00001F076FD094B0193029400964FF480734E
:1014F00004F52172294604F1440001F04FFE04B0C6
:1015000070BD00BF6C370008AD140008D11300088F
:101510000B68202282F311880A7903EB82021062A1
:101520004A790D3243F822008A7912B103EB820323
:10153000186202230372C0F88C14002383F311880D
:101540007047000038B5044601250221043001F03F
:10155000A7FC04F10C0025756FF00101FFF756FEA2
:1015600084F84C5004F144006FF00101BDE83840AC
:10157000FFF74CBE10B501210446043001F090FC89
:101580000023237584F84C3010BD000038B50446A4
:1015900000250C3001F034FD04F14400257501F004
:1015A00015FE201D84F84C50012101F079FC2046E5
:1015B000BDE83840FFF756BF90F85C3003F0600399
:1015C000202B19D190F85D20212A0AD0222A4FF031
:1015D00000030ED0202A0FD1084A02650722426577
:1015E00004E0064B03650723436500238365012060
:1015F000704703654365F9E700207047240802201F
:10160000D0F88C3437B51A681178042904461AD1F9
:10161000017A022917D11979128901238B401342CB
:1016200011D100F14405284601F0A6FE58B101A9E8
:10163000284601F0D7FDD4F88C44019B217902465D
:10164000206800F0CFF803B030BD000000EB81034C
:10165000F7B51C6A05460E46F4B1202383F31188C2
:1016600005EB8607201D082101F01AFCFB685B6969
:101670001B68443413B1204601F0C2FD01A9204685
:1016800001F0B0FD024648B1019B3146284600F00A
:10169000A9F8002383F3118803B0F0BDFB685A69F1
:1016A0001268002AF5D01B8A013B1340F1D105F1E5
:1016B0005C02EAE70D3110B550F82140CCB120238F
:1016C00083F311880421601801F0EAFBD4F88C241C
:1016D0001368527903EB820304F10C00DB689B6909
:1016E000596801F0A3FC2046FFF7BCFE002383F3FA
:1016F000118810BD7047000000F0F4BF4FF0804328
:10170000002258631A610222DA6070474FF080436A
:101710000022DA60704700004FF080435863704742
:1017200000F0A4BB012303700023436000F12402F6
:1017300000F1380142F8043B8A421361FAD1038177
:101740004381704738B50446202383F31188002570
:101750004160C560056145618561C561056200F054
:10176000A1FB0223237085F3118838BD70B500EB0F
:10177000810305465069DA600E46144618B11022FE
:10178000002101F03DFFA06918B11022002101F0F5
:1017900037FF31462846BDE8704000F05DBC0000D0
:1017A000028902F001020281428902F001024281B3
:1017B0000022026142618261C261026200F0E0BC0B
:1017C000F0B400EB81044789E4680125A4698D40E9
:1017D0003D43458123600023A2606360F0BC00F0BC
:1017E000FBBC0000F0B400EB81040789E46801252C
:1017F00064698D403D43058123600023A2606360DE
:10180000F0BC00F079BD000070B50223002504464D
:101810000370A0F8645080F8665080F86750058126
:101820004581C560056145618561C561056280F8D6
:101830004C5000F0AFFB63681B6823B1294620467B
:10184000BDE87040184770BD436802781B6880F897
:101850006820052202700BB1042118477047000070
:10186000436890F868201B6802700BB10521184787
:101870007047000070B50023044680F84C3000F13A
:101880005C0200F09FFC63689B685BBB94F85C5053
:1018900015F0600614D194F85D3005F07F0545EA37
:1018A0000325B5F5407F00F0A58059D8022D00F042
:1018B000F1803FD8002D00F08780012D00F0E480FA
:1018C0000021204600F0DCFE0021204600F0CEFE84
:1018D00063681B6813B1062120469847062384F8E5
:1018E0004C3070BD204698470028CFD094F8632034
:1018F00094F8623043EA0223626D934238BF636515
:1019000094F95C30656D002B4FF0200380F201816B
:10191000002D00F0F080012284F84C2083F3118820
:101920000021636D226D2046FFF75CFF002383F3E7
:10193000118870BDB5F5807F4DD0B5F5817FBFD1E1
:1019400094F85E30002BBBD194F8603013F00F0197
:1019500026D01A06204640F1B78000F0A5FE1FE011
:10196000B5F5C06F50D020D840F202339D4200F050
:10197000AE80B5F5A06FA3D1B4F85C30B3F5A06F1D
:101980000ED194F85E3084F86630204600F058FBA3
:1019900063681B6813B10121204698470323237015
:1019A000002323656365A365A0E7B5F5106F41D0FB
:1019B00040F602439D4267D0B5F5006F80D104F137
:1019C00067032365012333E004F1640323650223E5
:1019D0006365A5658AE794F85E30012B7FF470AFEC
:1019E000B4F8643023F00203A4F864302665666519
:1019F000A6657BE794F85E30012B7FF461AFB4F805
:101A0000643043F00203EFE794F86120616894F8D2
:101A100060304D6894F85F1043EA0223204694F842
:101A20005E20A84700283FF44BAF43682365036856
:101A30006365DDE794F8672094F85E309A42AFD092
:101A40002378042B10D1202383F311882046FFF73D
:101A5000A7FE86F31188636884F867601B6803211A
:101A600021700BB12046984794F85E30002B97D038
:101A700084F867300423237063681B68002B8FD0C1
:101A80000221204698478BE72E4B2365022363658E
:101A9000002388E794F8601011F0800F204601F0D1
:101AA0000F010ED000F080FB012806D002287FF441
:101AB00007AF254B236560659AE7244B2365656571
:101AC00096E700F063FBEFE700F0E4FD68E794F8C9
:101AD0005E30002B7FF4F4AE94F8603013F00F0109
:101AE0003FF45EAF1B06204602D500F0C9FD57E764
:101AF00000F0BCFD54E7032284F84C2083F31188E6
:101B00002B462A4629462046FFF75AFE85F31188C0
:101B100070BD5DB1042284F84C2083F3118800214C
:101B2000636D226D2046FFF74BFEFFE6052284F829
:101B30004C2083F311882B462A4629462046FFF77E
:101B400051FEE3E7943700088C370008903700080F
:101B500038B590F84C300446062B22D8DFE803F065
:101B6000370422373732370090F8631090F862203C
:101B7000436D42EA01229A4214D9C268128AB3FB29
:101B8000F2F502FB15356DB9202383F311882B463E
:101B90002A462946FFF726FE85F31188022384F89A
:101BA0004C3038BD032384F84C30202383F3118854
:101BB00000231A4619462046FFF702FE002383F34E
:101BC000118838BD836D03B198470023E7E70021F2
:101BD00000F056FD0021204600F048FD63681B68B8
:101BE00013B10621204698470623D8E790F84C20E9
:101BF000062A38B5044621D80123934013F0670F15
:101C00001DD113F008050FD1DB0617D5052380F889
:101C10004C30202383F311882B462A462946FFF7B0
:101C2000E1FD85F3118838BDC3689B695B682BB9FA
:101C3000836D03B19847002384F84C3038BD0021F0
:101C400000F01EFD0021204600F010FD63681B68B7
:101C500013B10621204698470623EDE7036F30B500
:101C600000229D68C46E11464FF0FF3004EB421312
:101C700001329542C3F80019C3F81019C3F80809D6
:101C8000C3F8001BC3F8101BC3F8080BEED24FF0CB
:101C90000113C4F81C3830BD890141F020010161F5
:101CA00003699B06FCD4122001F008B82DE9F04F1F
:101CB000202387B00446C56E83F3118800F17C03AE
:101CC00005934FF0000B2378012B04D0A36F4BB981
:101CD0006B69DB0606D4AB69059843F01003AB6172
:101CE000FFF760FA8BF311884FF0000E4FF02009D8
:101CF000236F9B685FFA8EF083421BD2202383F30D
:101D00001188E0E7E16E0A6A02F4F013B3F5802F60
:101D100066D0B3F5402F0DD1C2F30A1602F00F02C0
:101D200004EB820201F58051D3681F6A00231A4632
:101D30009E4248D1696911F01001E3D1012303FAF1
:101D400000F2A36F1A4200F08C8089F31188AB680F
:101D500023F00103AB60A36F23EA0203A36781F3BF
:101D6000118804EB8003D3F80C80D8F814100B68AA
:101D70000093431C1B030293430104934868009B98
:101D800098425FD2B8F81060E76E1B1AB34228BFC2
:101D90003346049EBE19D6F81869B6B2B3EB860F67
:101DA00062D8029EBE1903968E680196A6F1040AB7
:101DB0009C46039E5AF8047F3760BCF1040F3BD960
:101DC000ACF1040CF5E713F0030F08BF0A68072B0A
:101DD00098BF3A7003F101039CBF120A0137A7E7CD
:101DE000C2F30A1602F00F0204EB820201F58051E1
:101DF000D3689B691F68D3F808805B68A7EB030C66
:101E000000231F469E4208D1D36899698A684B68AF
:101E1000324433448A604B608CE713F0030F08BFF1
:101E20000F689C4588BF88F8007003F1010384BFE8
:101E30003F0A08F10108E5E7019E1E4403448E6055
:101E40004B609BE7012189F31188AB6843F00103E4
:101E5000AB6021B9D5F834381A43C5F834288BF370
:101E600011880EF1010E43E70021ECE710B50B4C91
:101E70002046FFF757FC4FF0A0420023E266084AD5
:101E80002267E367C4F8803004F5467104F18800E6
:101E90005522BDE81040FFF711B900BF600E0220C7
:101EA000BC37000870B50378012B86B005465DD1BC
:101EB000304BC46E984213D12F4B5A6B42F08002C4
:101EC0005A635A6942F080025A6100225A610E2117
:101ED000432001F071FA294BE360294BC4F8003824
:101EE0000023AB67C4F8003EC02323604FF4041303
:101EF000A363EE6E202000F0E1FE0123336133691D
:101F0000DB07FCD4122000F0D9FE3369002BFCDA89
:101F10000026A6602846FFF7A1FE6B68C4F810688B
:101F2000DB68C4F81468C4F81C680BBB154BA361CC
:101F30004FF0FF336361D5F880309BB9124B0093AB
:101F400005F18803019305F5467302930223039379
:101F500068460E4B04930595FFF7D0F8C5F880004E
:101F6000FFF782F8A36843F00103A36006B070BDD9
:101F7000074BDCE7600E02200038024040140040AE
:101F800003002002003C30C0C8370008AD1C000828
:101F9000083C30C0F8B5C46E054600212046FFF766
:101FA0007BFE296F00234FF001128F68C4F834388C
:101FB0004FF00066C4F81C284FF0FF3004EB4312CA
:101FC00001339F42C2F80069C2F8006BC2F80809E9
:101FD000C2F8080BF2D20B686B676362EB6E1022DB
:101FE0001A611E6916F01006FBD1122000F066FE81
:101FF000D4F8003823F4FE63C4F80038A36943F42E
:10200000402343F01003A3610923C4F81038C4F837
:102010001438094BEB60094BC4F8106BC4F8003B53
:10202000C4F81069C4F800396B6F03F1100243F46F
:1020300080136A67A362F8BD9837000840800010DB
:10204000C26E90F86610D2F8003823F4FE6343EABB
:102050000113C2F8003870472DE9F0410EB200EBD1
:1020600086080D46D8F80C100F6807F00303022B02
:1020700050D0032B50D03D4A3D4F012B18BF17467F
:10208000C46E4FEA451E04EB0E030022C3F8102B6A
:102090008A6905F1100C002A40D04A8A05F15803DC
:1020A0005B013A43E2500123D4F81C2803FA0CF3F5
:1020B0001343A6444A69C4F81C380023CEF81039EB
:1020C00005F13F03002A39D00A8A898B9208012939
:1020D00088BF4A43416F04EB8303561841EA02422A
:1020E000466729465A602046FFF7D6FDD8F80C30DF
:1020F0001B8A43EA85531F4305F148035B01E75000
:102100000123D4F81C2803FA05F51543C4F81C581C
:10211000BDE8F081174FB3E7174FB1E704EB461363
:10212000D3F8002B22F40042C3F8002BD4F81C286B
:10213000012303FA0CF322EA0303BAE704EB830357
:102140000E4A5A6004EB461629462046FFF7A4FDC6
:10215000D6F8003923F40043C6F80039D4F81C3807
:10216000012202FA05F523EA0505CFE700800010F9
:10217000008004100080081000800C100004000291
:10218000026F12684267FFF769BD00005831C36EE5
:1021900049015B5813F4004004D013F4001F14BF2E
:1021A00001200220704700004831C36E49015B588E
:1021B00013F4004004D013F4001F14BF01200220C8
:1021C0007047000000EB8101CB68196A0B6813604F
:1021D0004B6853607047000000EB810330B5DD6849
:1021E000AA691368D36019B9402B84BF40231360D8
:1021F0006B8A1468C26E1C44013CB4FBF3F4634365
:10220000033323F0030302EB411043EAC44343F0DA
:10221000C043C0F8103B2B6803F00303012B09B245
:102220000ED1D2F8083802EB411013F4807FD0F8B9
:10223000003B14BF43F0805343F00053C0F8003B11
:1022400002EB4112D2F8003B43F00443C2F8003BDA
:1022500030BD00002DE9F041264DEE6E06EB401337
:102260000446D3F8087BC3F8087B38070AD5D6F8AC
:102270001438190706D505EB84032146DB68284688
:102280005B689847FA0733D5D6F81438DB072FD5A3
:1022900014B995F84C305BB305EB8403D968CCB91D
:1022A0008B69488A5E68B6FBF0F200FB12628AB95D
:1022B0001868DA6890420DD2121A83E814002023BD
:1022C00083F311880B482146FFF786FF84F31188BA
:1022D000BDE8F081012303FA04F26B8923EA0203CB
:1022E0006B81CB6823B121460248BDE8F041184715
:1022F000BDE8F081600E022000EB810370B5DD685F
:10230000C36E6C692668E6604A0156BB1A444FF4F6
:102310000020C2F810092A6802F00302012A0AB25A
:102320000ED1D3F8080803EB421410F4807FD4F8E0
:10233000000914BF40F0805040F00050C4F800097C
:1023400003EB4212D2F8000940F00440C2F8000941
:10235000D3F83408012202FA01F10143C3F834181A
:1023600070BD19B9402E84BF4020206020682E8A9D
:10237000841940F00050013C1A44B4FBF6F440EAE2
:10238000C440C6E72DE9F041284CE66E06EB401349
:102390000546D3F80879C3F80879F9071AD5D6F8AD
:1023A0001038DA0716D504EB8003D9684B69186832
:1023B000DA6890422CD2121A4FF000081A60C3F863
:1023C0000480202383F3118829462046FFF794FFD9
:1023D00088F311883B0619D5D6F83428012303FA6F
:1023E00005F5154212D0202383F31188A36F1048FE
:1023F0002B43A367D6F8343823EA0505C6F83458CA
:102400000021FEF7DDFE002383F31188BDE8F08193
:10241000012303FA05F2238923EA020323818B684F
:10242000002BD7D0294620469847D3E7600E0220DC
:10243000DC0E02202DE9F74F8A48C46E6669A36955
:102440001E4016F4805F6661054608D0002383674E
:10245000FFF7DAF903B0BDE8F04F00F079BD002EC8
:1024600012DAD4F8003E7F4899071EBFD4F8003E28
:1024700023F00303C4F8003ED4F8043843F001030A
:10248000C4F80438FFF7ECF9320504D50023754889
:10249000AB67FFF7D9F9B3040CD5D4F8083813F0BB
:1024A000060FE36823F470530CBF43F4105343F456
:1024B000A053E360370704D56B68DB680BB169484C
:1024C0009847F00262D4B1020CD5D5F86C80DFF8E1
:1024D00094A100274FF001092B6F9B68F9B28B4242
:1024E00080F0A380F2060DD5202383F31188A36921
:1024F0005D4823F01003A3610021FEF761FE002375
:1025000083F311883303D4F818481DD5E70302D5A7
:102510000020FFF79FFEA50302D50120FFF79AFEDA
:10252000600302D50220FFF795FE210302D50320A8
:10253000FFF790FEE20202D50420FFF78BFEA30214
:1025400002D50520FFF786FE770383D5E60702D57F
:102550000020FFF717FFA50702D50120FFF712FFA4
:10256000600702D50220FFF70DFF210702D50320E7
:10257000FFF708FFE20602D50420FFF703FFA306DA
:102580007FF568AF0520FFF7FDFE63E7D5F86CA087
:10259000DFF8D4B04FF000092B6F9B685FFA89F722
:1025A000BB4290D30AEB4713D3F8002902F4402230
:1025B000B2F5802F36D1D3F80029002A32DAD3F8C9
:1025C000002942F09042C3F80029D3F80029002ADC
:1025D000FBDB3946E86EFFF75FFB01232A89BB402E
:1025E0006FEA030808EA02022A8105EB8702D26833
:1025F000926822B139461B4801939047019B2022E3
:1026000082F31188DAF8342808EA0202CAF834287A
:10261000AA6F002113435846AB67FEF7D1FD002394
:1026200083F3118809F10109B6E708EB4112D2F8EA
:10263000003B03F44023B3F5802F10D1D2F8003BC8
:10264000002B0CDA6A8909FA01F322EA03036B8191
:1026500005EB8103DB68DB680BB150469847013717
:102660003AE700BF600E0220DC0E0220C36E03EBCF
:102670004111D1F8003B43F40013C1F8003B70470F
:10268000C36E03EB4111D1F8003943F40013C1F8D4
:1026900000397047C36E03EB4111D1F8003B23F4BE
:1026A0000013C1F8003B7047C36E03EB4111D1F832
:1026B000003923F40013C1F8003970474FF080430C
:1026C00010B51A69920708D500241C61202383F3F2
:1026D000118800F0B9FA84F31188BDE8104000F0C9
:1026E00037BC00000E4A136C43F0010313640D4A1B
:1026F000936843F0010393604FF080436B229A622A
:102700004FF0FF32DA6200229A615A63DA605A604F
:1027100001225A6108211A601C2000F04DBE00BF42
:1027200000380240002004E000207047FEE700006F
:10273000704700004FF0FF307047000000F07CBE93
:1027400008B500F033FC00F033FABDE8084000F0B3
:10275000FFB8000070470000022906D0032906D008
:102760000129064818BF0020704705487047032A12
:102770009ABF044800EBC20000207047143A0008DA
:10278000C83900082C08022070B5044608460D46DA
:10279000FDF7DAFDC6B22046013403780BB91846BE
:1027A00070BD3246294600F079FF0028F3D10120A0
:1027B00070BD00002DE9F84F804608460F46FDF732
:1027C000C3FD3E49C4B23846FFF7DEFF08B104340A
:1027D000E4B23B493846FFF7D7FF08B11034E4B202
:1027E000601C00F0C3F9DFF8E490DFF8E4B0824643
:1027F00004463D462E780EBB26705046FDF7A4FDDC
:10280000C5B26C1C64002146C8F80040012000F0ED
:10281000C5F90322C8F80400047042705146023022
:10282000A1EB0A02D2B2954200F102003DD8574511
:1028300042D05046BDE8F84F00F0B4B9252E30D153
:102840001E492846FEF7E2F970B9DBF80010216056
:10285000DBF804106160BBF8081021819BF80A10B6
:10286000A17207350B34C5E715492846FEF7CEF9A6
:10287000B8B9144EA11C16F8010F134B4FEA101EE5
:1028800000F00F001EF809E010F8090001F802EC52
:102890009E4201F8010C01F10201ECD11834083517
:1028A000A8E7267001350134A4E711F8012B00F8E0
:1028B000022C00F8016CB3E7BDE8F88F5839000826
:1028C000603900081FF4F01F2BF4F01F7539000861
:1028D0006939000808B5202383F311880348FEF7FF
:1028E0008FFE002383F3118808BD00BF90110220E2
:1028F00010B50446052916D8DFE801F016150316B1
:10290000161D202383F311880E4A0121FEF72EFFA6
:1029100020460D4A0221FEF729FF0C48FEF736FE3D
:10292000002383F3118810BD202383F31188074807
:10293000FEF708FEF4E7202383F311880348FEF72F
:1029400019FEEDE7083900082C3900089011022023
:1029500010B5094C094904F10800FFF72BFF04F1F9
:1029600010000749FFF726FF04F118000549BDE8EC
:102970001040FFF71FBF00BF2C0802208839000855
:102980009F39000860390008024AD368DB03FCD491
:10299000704700BF003C024008B5FFF7F5FF054B4C
:1029A0001A69002ABFBF044A5A6002F188325A608D
:1029B00008BD00BF003C02402301674508B5FFF792
:1029C000E3FF034A136943F00043136108BD00BFEE
:1029D000003C02400B2870B513D80B4A0B4C1378FF
:1029E00063B90B4E4FF0006144F8231056F82350A2
:1029F00001330C2B2944F7D10123137054F8200024
:102A000070BD002070BD00BF80160220501602204D
:102A1000343A0008014B53F820007047343A00085C
:102A20000C2070470B2810B5044601D9002010BDBA
:102A3000FFF7AAFFFFF7B0FF1449F320C860FFF7C4
:102A4000A3FFE300DBB243F4007343F002030B6126
:102A50000B6943F480330B61FFF796FFCB681BB122
:102A6000C860FFF7ABFFE1E7FFF7A8FF2046FFF7DD
:102A7000B1FF074B53F824300344834201D10120B6
:102A800010BD0278FF2AD1D10130F6E7003C0240A8
:102A9000343A0008F8B51646F20738D43318B3F1C3
:102AA000026F34D21F4B1B68DB0730D51E4CFFF77B
:102AB00073FFF323E360FFF767FF236923F4407399
:102AC0002361236943F4807343F0010323610F46BC
:102AD000401AF31BD94200EB070507D1236923F005
:102AE00001032361FFF76AFF3046F8BD37F8023B68
:102AF0002B80BFF34F8FFFF747FFE36853B1F323FA
:102B0000E360236923F001032361FFF757FF4FF0D0
:102B1000FF30F8BD2D8837F8023CADB2AB42D8D0BB
:102B2000EFE700BF00380240003C024038B50D4BD3
:102B30001A78044642B901221A704FF000514FF43E
:102B400000320948FEF77EFB082221460648FEF7C0
:102B500085FB054618B12246002100F051FD2846AC
:102B600038BD00BFA81602208816022038B50446DA
:102B700088B1014608220020FEF770FB054628B107
:102B80002246002100F03CFD284638BD2046BDE825
:102B90003840FFF7CBBF0546F6E700004843FFF794
:102BA000E5BF000008B1FEF7CFBB7047FEE70000AD
:102BB00010B51D4CFEF79AF9FEF714F900F0BAF8BB
:102BC00000F082F9FEF730FB802218492046FEF71C
:102BD00055FA012380F82030154B164AD96844F87D
:102BE000180C21F4E0610904090C0A43002412497D
:102BF000C461DA60CA6842F08072CA600F4A104944
:102C0000C2F8B01F116841F0010111601022DA779B
:102C1000202283F8222084F3118862B60948BDE897
:102C20001040FEF773BA00BFF80D0220843A000886
:102C300000ED00E00003FA05F0ED00E0001000E018
:102C400055CEACC5643A00082DE9F8431A4C4FF054
:102C500080430025E769586A04F11C082E46A26AE1
:102C6000BB68811A8B420CD9E169414522D01344DB
:102C70001B1A022B2CBFC0180230BDE8F843FEF728
:102C80004BBD1344A3623B68D7F80C90C3F8048093
:102C90004345E361FD6001D1FEF738FD86F31188FD
:102CA0003869C847202383F311884FF08043E769D0
:102CB000586AD4E7BDE8F883C80D0220034B596871
:102CC0005A68521A9042FBD8704700BF001000E0CB
:102CD0004FF0FF330360002343608360C360002232
:102CE0000023C0E904237047014B5B688360704791
:102CF000001000E00D4A0E4B516FC2685B68013254
:102D0000C260826830B5D0E904459B1A5B1A4268FC
:102D10008360E41845F100059342026888BF436070
:102D20009342C0E9044538BF036030BDC80D02209E
:102D3000001000E010B5084C86B0002368466367B9
:102D4000FFF7C6FF6846FFF7CFFF6846FFF7D2FFE1
:102D5000029B636706B010BDC80D022010B50B467C
:102D60001B68994205D15A68036042601060586040
:102D700010BD9C6882689442F2D2F4E700230060A0
:102D8000406083607047000070B51E4B84689D6989
:102D900006467CB9AB6B8560C360A86370BD94E8E0
:102DA0000C001A6022685360616A2046FFF7D6FF64
:102DB000636A9C68AB68A2689A4219D2A36094F8CF
:102DC0002030062BEBD0072B09D08BB994E80C00F0
:102DD0001A60226820465360FEF792F808E094E8F3
:102DE0000C001A6022685360616A2046FFF7B6FF44
:102DF00028463146FFF7B2FF6E620620BDE87040FC
:102E0000FEF7C6B8C80D022008B5202383F3118849
:102E1000FFF7BAFF002383F3118808BD144A38B5C1
:102E200091690346202282F31188C26800688A6390
:102E300098421AD0CC6B7AB902688C601A605360E1
:102E4000826B9860DA608363FEF75AF8FEF70CF93C
:102E5000002383F3118838BD1568AA4203D0AD68FA
:102E6000AC4238BF2C46D268E5E700238360EFE729
:102E7000C80D0220436B194390F8203041630A2BA0
:102E800003D1436A194205D170470B2B06D1436A1F
:102E90008B4303D100234362FEF732B87047000032
:102EA00070B5046805460E46AC4200D170BDE368BB
:102EB0003343E36016B12269134203D0A16860680E
:102EC000FFF7D8FF2468EFE7034B044A1A60044B6E
:102ED000044A1A60704700BFD4180220D818022094
:102EE000D01802200000082030B5094C2368421E8B
:102EF000581E084B4D4208441B6828400A442A408B
:102F00001B1A9A429ABF12182260002030BD00BFDF
:102F1000D4180220D018022008B5202383F311888A
:102F2000FFF7E2FF002383F3118808BD80B5074A4D
:102F3000536823F0010300AF5360EFF30983683354
:102F400083F30988002383F3118880BD30EF00E00C
:102F500098B5202300AF83F31188104B5B6813F4FE
:102F6000006318D0F1EE103AEFF309844FF080734C
:102F700044F84C3C0A4BDB6844F8083CA4F1680375
:102F800083F30988FEF74EF818B1064B44F8503C1D
:102F900098BD054BFAE783F3118898BD00ED00E07A
:102FA00030EF00E0410300084403000808B500F0DA
:102FB00019FA064800F0C8FAFEF7B2FBFEF77AFAF3
:102FC000FFF7C8FBBDE80840FEF796BBD437000802
:102FD00030B5039C0172043304FB0325C361049BD9
:102FE00003630021059B00604060C1604261026193
:102FF0008561046242628162C162436330BD000048
:103000000022416A41610161C2608262C2626FF066
:103010000101FEF7FBB8000003694269934203D146
:10302000C2680AB100207047181D70470369196013
:10303000C2680132C260C26913448269036193426B
:1030400024BF436A03610021FEF7D4B838B50446B3
:103050000D46E3683BB16269131D1268A362134415
:10306000E362002038BD237A33B929462046FEF7B3
:10307000B1F80028EDDA38BD6FF00100FBE7000081
:10308000C368C269013BC3604369134482694361F9
:10309000934224BF436A436100238362036B03B1FD
:1030A0001847704770B52023044683F31188866A59
:1030B0003EB9FFF7CBFF054618B186F311882846C5
:1030C00070BDA36AE26A13F8015BA362934202D364
:1030D0002046FFF7D5FF002383F31188EFE70000B8
:1030E0002DE9F74F1F4604460E469146202383F3F1
:1030F00011884FF080480025D8F82430FB18009341
:1031000007F1FF3AAB46A36AABB91AF1030F06D930
:1031100039462046FFF79AFF68B1002305E0D8F84A
:103120002410009A511A8F42F3D283F31188284653
:1031300003B0BDE8F08FA16AE36AA9EB05025B1A50
:10314000934228BF1346402B1CD9334601F140025D
:1031500051F8040B43F8040B9142F9D1A36A4033B0
:103160004036A3624035A26AE36A9A4202D32046FF
:10317000FFF786FF8BF311884D45D8D2202383F3C8
:103180001188C0E71A4630460193FDF735FD019BD3
:10319000A26A1A441E44A2621D44E4E710B5029CD0
:1031A0000172043303FB0421C36100238362C36201
:1031B000039B0363049B00604060C4604261026142
:1031C000816104624262436310BD0000026AC26012
:1031D000426A4261026100228262C2626FF00101B2
:1031E000FEF714B8436902699A4203D1C2680AB172
:1031F00000207047184650F8043B0B6070470000F1
:10320000C368C2690133C36043691344826943617F
:10321000934224BF436A43610021FDF7EBBF0000E6
:1032200038B504460D46E3683BB123691A1DA26216
:10323000E2691344E362002038BD237A33B929469A
:103240002046FDF7C7FF0028EDDA38BD6FF001001A
:10325000FBE7000003691960C268013AC260C269F5
:10326000134482690361934224BF436A03610023CC
:103270008362036B03B118477047000070B52023C9
:1032800004460E4683F31188856A35B91146FFF767
:10329000C7FF10B185F3118870BDA36A1E70A36AC1
:1032A000E26A01339342A36204D3E1692046043900
:1032B000FFF7D0FF002080F3118870BD2DE9F74F94
:1032C0001F4604460D469146202383F311884FF094
:1032D00080480026D8F82430FB18009307F1FF3A05
:1032E000B346A36AABB91AF1030F06D93946204693
:1032F000FFF796FF68B1002305E0D8F82410009A84
:10330000511A8F42F3D283F31188304603B0BDE8DF
:10331000F08FA06AE36AA9EB06021B1A934228BF4A
:103320001346402B1CD905F1400355F8042B40F8F7
:10333000042B9D42F9D1A36A4033A3624036A26AAE
:10334000E36A9A4204D3E16920460439FFF782FF19
:103350008BF311884E45D8D2202383F31188C0E720
:103360001A4629460193FDF747FC019BA26A1A44BD
:103370001D44A2621E44E2E7026943699A4203D1F6
:10338000C3681BB9184670470023FBE7836A002B0C
:10339000F8D0043B9B1AF5D01360C368013BC360AF
:1033A000C3691A44836902619A4224BF436A036174
:1033B000002383620123E5E700F1604300F01F0270
:1033C000400903F5614309018000C9B200F1604082
:1033D00083F8001300F5614001239340C0F8803169
:1033E00003607047124B00211A694FF0FF321A61D7
:1033F000196158695A615961186A60F08050186201
:103400001962586A5A620B4A5962106840F4807017
:103410001060186F00F44070B0F5007F1EBF4FF4CD
:10342000803018671967536823F40073536070473E
:103430000038024000700040354B364A1A64364A64
:103440004FF4404111601A6842F001021A601A6894
:103450009207FCD59A6822F003029A609A689A60F3
:103460002B4B19469A6812F00C02FBD1186800F039
:10347000F90018609A601A6842F480321A600B688A
:103480009B03FCD54B6F43F001034B67204B5A6FF6
:103490009007FCD5214A5A601A6842F080721A607F
:1034A0001D4B1A4659684904FCD5196841F480310E
:1034B00019605368D803FCD5136843F400331360D4
:1034C000154A53689903FCD5114B1A689201FCD533
:1034D000134A9A6040F20112C3F88C200022C3F80C
:1034E0009020104A40F2093111609A6842F00202BD
:1034F0009A60074B9A6802F00C02082AFAD15A6CBB
:1035000042F480425A645A6E42F480425A667047CE
:10351000003802400004001000700040186C4009A0
:1035200000948838003C02404B6843608B6883609D
:10353000CB68C3600B6943614B6903628B6943626B
:103540000B68036070470000214B0246186B10B5F2
:1035500040F2FF7420431863196D1E48214319651A
:103560001146FFF7E1FF1C4802F11C01FFF7DCFFE9
:103570001A4802F13801FFF7D7FF194802F1540148
:10358000FFF7D2FF174802F17001FFF7CDFF164891
:1035900002F18C01FFF7C8FF144802F1A801FFF700
:1035A000C3FF134802F1C401FFF7BEFF114802F147
:1035B000E001FFF7B9FF104802F1FC01FFF7B4FF8B
:1035C0000E4802F58C71BDE81040FFF7ADBF00BF9B
:1035D000003802400000024000040240000802409F
:1035E000000C02400010024000140240001802408B
:1035F000001C02400020024000240240002802403B
:1036000070B4860746D0541E002A41D0CAB2034681
:1036100002E014F1FF343BD303F8012B9D07F8D1EE
:10362000032C2ED9CDB245EA05250F2C45EA0545D8
:1036300019D903F110022646103E0F2E42F8105CF5
:1036400042F80C5C42F8085C42F8045C02F110029B
:10365000F2D8A4F1100222F00F0204F00F0410328D
:10366000032C13440DD91E462246043A032A46F879
:10367000045BFAD8221F22F003020432134404F040
:1036800003042CB1C9B21C4403F8011B9C42FBD1BA
:1036900070BC704714460346C2E700BF002A41D001
:1036A00040EA010313F00303F0B425D1032A23D920
:1036B00004680D68AC421FD1043A38D0A4F101353A
:1036C00025EA040414F0803F2ED1043004310FE0C9
:1036D00050F8043B0E68A3F10134B34224EA03041A
:1036E00001F1040126D1043A21D014F0803F1BD10E
:1036F000032A07460D46EBD805780C78AC4202F158
:10370000FF331AD183B114B90EE06BB17AB110F85E
:10371000012F11F8014FA24203F1FF33F5D0101B26
:10372000F0BC7047104670470020F0BC7047104650
:10373000F0BC704729463846DEE72A46EFE700BF6F
:1037400053544D3332463F3F3F3F3F3F0053544D6C
:10375000333246375B347C355D780053544D333219
:1037600046375B367C375D78000000003114000876
:103770001D140008591400084514000851140008CD
:103780003D1400082914000815140008000000006A
:103790000100000000000000000000007518000893
:1037A000511B0008ED1B000840004000781102206A
:1037B0007811022001000000881102208000000022
:1037C00040010000050000007573625F70756D7048
:1037D000000000000000802A00000000AAAAAAAA97
:1037E00000000000FFFF00000000000000A00A0031
:1037F0000000000000000000AAAAAAAA0000000021
:10380000FFFF0000000000000000000000000000BA
:1038100000000000AAAAAAAA00000000FFFF000002
:103820000000000000000000000000000000000098
:10383000AAAAAAAA00000000FFFF000000000000E2
:10384000000000000000000000000000AAAAAAAAD0
:1038500000000000FFFF000000000000000000006A
:103860000000000000000000AAAAAAAA00000000B0
:10387000FFFF00000000000000000000000000004A
:1038800000000000AAAAAAAA00000000FFFF000092
:103890000000000000000000000000000000000028
:1038A000AAAAAAAA00000000FFFF00000000000072
:1038B000000000000000000000000000AAAAAAAA60
:1038C00000000000FFFF00000000000000000000FA
:1038D00000000000000000000000000000000000E8
:1038E00000000000000000000000000000000000D8
:1038F00000000000000000000000000000000000C8
:1039000000000000000000000200000000000000B5
:103910004D160008B5160008400040002016022091
:10392000301602200200000000000000030000002A
:1039300000000000F5160008000000001000000064
:1039400040160220000000000100000000000000FE
:10395000600E02200101020025424F415244250021
:103960002553455249414C2500637562652D6F72A0
:10397000616E67650030313233343536373839415E
:10398000424344454600000048657820546563681A
:103990006E6F6C6F6779204C696D69746564005057
:1039A000726F6669434E432043554245204F726112
:1039B0006E676520424C0000F12800085927000876
:1039C000B9150008D528000843000000D0390008C8
:1039D00009024300020100C0320904000001020292
:1039E0000100052400100105240100010424020245
:1039F0000524060001070582030800FF09040100F1
:103A0000020A0000000705010240000007058102CC
:103A100040000000120000001C3A000812011001D2
:103A200002000040AE2D011000020102030100005F
:103A300004030904008000000080000000800000F2
:103A400000800000000002000000040000000400EC
:103A50000000040000000400000004000000040056
:103A6000000004007C3A0008B0160220D0180220A2
:103A700001000000AD2B00080000000069646C65C7
:103A8000000000006D61696E001600200404440807
:103A90000C1014181C20212200000000000000005F
:103AA00000000000403700083F000000490400000B
:103AB0004D3700083F000000510400005B3700084C
:103AC0003F00000000960000000008000400000015
:103AD000303A000800000000000000000000000074
:0C3AE000000000000000000000000000DA
:00000001FF
